:020000040800F2
:1000000000060020E1020008E3020008E302000805
:10001000E3020008E3020008E3020008E30200082C
:10002000E3020008E3020008E3020008B128000828
:10003000E3020008E3020008E3020008E30200080C
:10004000E3020008E3020008E3020008E3020008FC
:10005000E3020008E30200081D3E0008493E0008D4
:10006000753E0008A13E0008CD3E0008BD10000806
:10007000E5100008111100083D1100086911000881
:1000800091110008BD110008E3020008E302000816
:10009000E3020008E3020008E3020008F93E00085A
:1000A000E3020008E3020008E3020008E30200089C
:1000B000E3020008E3020008E3020008E30200088C
:1000C000E3020008E3020008E3020008E30200087C
:1000D000E3020008E3020008E3020008E30200086C
:1000E0005D3F0008E3020008E3020008E3020008A5
:1000F000E3020008E3020008E3020008E911000837
:10010000E3020008E3020008D13F0008E302000810
:10011000E3020008E3020008E3020008E30200082B
:10012000151200083D120008691200089512000817
:10013000C1120008E3020008E3020008E30200081D
:10014000E3020008E3020008E3020008E3020008FB
:10015000E91200081513000841130008E302000823
:10016000E3020008E3020008E3020008E3020008DB
:10017000E30200089D340008E3020008E3020008DF
:10018000E3020008E3020008E3020008E3020008BB
:10019000E3020008E3020008E3020008E3020008AB
:1001A000E3020008E3020008E3020008E30200089B
:1001B000E3020008E3020008E3020008E30200088B
:1001C000E3020008E3020008E3020008E30200087B
:1001D000E302000889340008E3020008E302000893
:1001E000E3020008E3020008E3020008E30200085B
:1001F000E3020008E3020008E3020008E30200084B
:10020000E3020008E3020008E3020008E30200083A
:10021000E3020008E3020008E3020008E30200082A
:10022000E3020008E3020008E3020008E30200081A
:10023000E3020008E3020008E3020008E30200080A
:10024000E3020008E3020008E3020008E3020008FA
:10025000E3020008E3020008E3020008E3020008EA
:10026000E3020008E3020008E3020008E3020008DA
:10027000E3020008E3020008E3020008E3020008CA
:10028000E3020008E3020008E3020008E3020008BA
:10029000E3020008E3020008E3020008E3020008AA
:1002A000E3020008E3020008E3020008E30200089A
:1002B000E3020008E3020008E3020008E30200088A
:1002C000E3020008E3020008E3020008E30200087A
:1002D000E3020008E3020008E3020008E30200086A
:1002E00002E000F000F8FEE772B6374880F30888B5
:1002F000364880F3098836483649086040F20000E5
:10030000CCF200004EF63471CEF200010860BFF36B
:100310004F8FBFF36F8F40F20000C0F2F0004EF637
:100320008851CEF200010860BFF34F8FBFF36F8F8B
:100330004FF00000E1EE100A4EF63C71CEF20001E3
:100340000860062080F31488BFF36F8F02F012FB61
:1003500003F020FB4FF055301F491B4A91423CBF30
:1003600041F8040BFAE71D49184A91423CBF41F895
:10037000040BFAE71A491B4A1B4B9A423EBF51F83D
:10038000040B42F8040BF8E700201849184A914280
:100390003CBF41F8040BFAE702F02AFB03F07EFBB6
:1003A000144C154DAC4203DA54F8041B8847F9E7A6
:1003B00000F042F8114C124DAC4203DA54F8041B21
:1003C0008847F9E702F012BB000600200022002057
:1003D0000000000808ED00E00000002000060020FA
:1003E000A8440008002200205C2200206022002097
:1003F000BC430020E0020008E0020008E002000820
:10040000E00200082DE9F04F2DED108AC1F80CD064
:10041000D0F80CD0BDEC108ABDE8F08F002383F338
:1004200011882846A047002001F0CAFDFEE701F030
:1004300059FD00DFFEE7000038B500F02FFC00F0AA
:10044000D1FD02F0F5F9054602F028FA0446C0B9DC
:100450000E4B9D4217D001339D4241F2883512BFA9
:10046000044600250124002002F0ECF90CB100F054
:1004700075F800F08BFD284600F01EF900F06EF8CC
:10048000F9E70025EFE70546EDE700BF010007B0FB
:1004900008B500F0D5FBA0F120035842584108BD33
:1004A00007B541F21203022101A8ADF8043000F0B3
:1004B000E5FB03B05DF804FB38B5302383F3118806
:1004C000174803680BB101F047FE0023154A4FF4AB
:1004D0007A71134801F036FE002383F31188124C21
:1004E000236813B12368013B2360636813B1636819
:1004F000013B63600D4D2B7833B963687BB90220F3
:1005000000F0A4FC322363602B78032B07D16368CF
:100510002BB9022000F09AFC4FF47A73636038BD67
:1005200060220020B90400088023002078220020E7
:10053000084B187003280CD8DFE800F00805020803
:10054000022000F071BC022000F05CBC024B0022D3
:100550005A6070477822002080230020F8B5504B65
:10056000504A1C461968013100F0998004339342C7
:10057000F8D162684C4B9A4240F291804B4B9B6899
:1005800003F1006303F500339A4280F08880002075
:1005900000F0AAFB0220FFF7CBFF454B0021D3F868
:1005A000E820C3F8E810D3F81021C3F81011D3F8ED
:1005B0001021D3F8EC20C3F8EC10D3F81421C3F8C1
:1005C0001411D3F81421D3F8F020C3F8F010D3F8A5
:1005D0001821C3F81811D3F81821D3F8802042F05D
:1005E0000062C3F88020D3F8802022F00062C3F8B4
:1005F0008020D3F88020D3F8802042F00072C3F826
:100600008020D3F8802022F00072C3F88020D3F835
:10061000803072B64FF0E023C3F8084DD4E90004EF
:10062000BFF34F8FBFF36F8F224AC2F88410BFF31E
:100630004F8F536923F480335361BFF34F8FD2F848
:10064000803043F6E076C3F3C905C3F34E335B0154
:1006500003EA060C29464CEA81770139C2F8747224
:10066000F9D2203B13F1200FF2D1BFF34F8FBFF32C
:100670006F8FBFF34F8FBFF36F8F536923F4003336
:1006800053610023C2F85032BFF34F8FBFF36F8F17
:10069000302383F31188854680F308882047F8BD0E
:1006A0000000020820000208FFFF010800220020CD
:1006B0000044025800ED00E02DE9F04F93B0B44B38
:1006C0002022FF2100900AA89D6800F009FCB14A91
:1006D0001378A3B90121B04811700360302383F36C
:1006E000118803680BB101F037FD0023AB4A4FF4CA
:1006F0007A71A94801F026FD002383F31188009B3D
:1007000013B1A74B009A1A60A64A1378032B03D0A3
:1007100000231370A24A53604FF0000A009CD34696
:100720005646D146012000F07FFB24B19C4B1B684C
:10073000002B00F02682002000F082FA0390039B39
:10074000002BF2DB012000F05DFB039B213B1F2B04
:10075000E8D801A252F823F0D907000801080008E0
:100760009508000825070008250700082507000848
:1007700027090008F70A0008110A0008730A000890
:100780009B0A0008C10A000825070008D30A0008D0
:1007900025070008450B0008790800082507000810
:1007A000890B0008E50700087908000825070008FC
:1007B000730A000825070008250700082507000818
:1007C0002507000825070008250700082507000859
:1007D00025070008950800080220FFF759FE0028A9
:1007E00040F0F981009B022105A8BAF1000F08BF73
:1007F0001C4641F21233ADF8143000F03FFA91E795
:100800004FF47A7000F01CFA071EEBDB0220FFF7B2
:100810003FFE0028E6D0013F052F00F2DE81DFE831
:1008200007F0030A0D1013360523042105A80593CC
:1008300000F024FA17E004215548F9E704215A484A
:10084000F6E704215948F3E74FF01C08404608F149
:10085000040800F04BFA0421059005A800F00EFAF8
:10086000B8F12C0FF2D101204FF0000900FA07F780
:1008700047EA0B0B5FFA8BFB00F07EFB26B10BF017
:100880000B030B2B08BF0024FFF70AFE4AE70421E5
:100890004748CDE7002EA5D00BF00B030B2BA1D1C1
:1008A0000220FFF7F5FD074600289BD00120002617
:1008B00000F01AFA0220FFF73BFE1FFA86F84046C6
:1008C00000F022FA0446B0B1039940460136A1F186
:1008D00040025142514100F027FA0028EDD1BA46BA
:1008E000044641F21213022105A83E46ADF8143029
:1008F00000F0C4F916E725460120FFF719FE244B46
:100900009B68AB4207D9284600F0F0F9013040F06F
:1009100067810435F3E70025224BBA463E461D7039
:100920001F4B5D60A8E7002E3FF45CAF0BF00B039C
:100930000B2B7FF457AF0220FFF7FAFD322000F0B7
:100940007FF9B0F10008FFF64DAF18F003077FF410
:1009500049AF0F4A08EB0503926893423FF642AF56
:10096000B8F5807F3FF73EAF124BB845019323DDCA
:100970004FF47A7000F064F90390039A002AFFF6AE
:1009800031AF039A0137019B03F8012BEDE700BF5C
:10099000002200207C23002060220020B9040008EF
:1009A000802300207822002004220020082200203A
:1009B0000C2200207C220020C820FFF769FD07469A
:1009C00000283FF40FAF1F2D11D8C5F120020AAB4C
:1009D00025F0030084494245184428BF424601924D
:1009E00000F058FA019AFF217F4800F079FA4FEAA7
:1009F000A803C8F387027C492846019300F078FADF
:100A0000064600283FF46DAF019B05EB830533E7F5
:100A10000220FFF73DFD00283FF4E4AE00F0A2F90C
:100A200000283FF4DFAE0027B846704B9B68BB42FE
:100A300018D91F2F11D80A9B01330ED027F00303BA
:100A400012AA134453F8203C05934046042205A9FA
:100A5000043700F01DFB8046E7E7384600F046F912
:100A60000590F2E7CDF81480042105A800F006F9FE
:100A700002E70023642104A8049300F0F5F800289D
:100A80007FF4B0AE0220FFF703FD00283FF4AAAECA
:100A9000049800F05DF90590E6E70023642104A8BE
:100AA000049300F0E1F800287FF49CAE0220FFF7E9
:100AB000EFFC00283FF496AE049800F04BF9EAE70B
:100AC0000220FFF7E5FC00283FF48CAE00F05AF955
:100AD000E1E70220FFF7DCFC00283FF483AE05A924
:100AE000142000F055F907460421049004A800F0F2
:100AF000C5F83946B9E7322000F0A2F8071EFFF624
:100B000071AEBB077FF46EAE384A07EB09039268FB
:100B100093423FF667AE0220FFF7BAFC00283FF48D
:100B200061AE27F003074F44B9453FF4A5AE4846F0
:100B300009F1040900F0DAF80421059005A800F095
:100B40009DF8F1E74FF47A70FFF7A2FC00283FF41C
:100B500049AE00F007F9002844D00A9B01330BD0BE
:100B600008220AA9002000F0C3F900283AD0202268
:100B7000FF210AA800F0B4F9FFF792FC1C4801F02D
:100B800025FA13B0BDE8F08F002E3FF42BAE0BF02A
:100B90000B030B2B7FF426AE0023642105A80593DD
:100BA00000F062F8074600287FF41CAE0220FFF731
:100BB0006FFC804600283FF415AEFFF771FC41F250
:100BC000883001F003FA059800F00AFA46463C46E0
:100BD00000F0D2F9A6E506464EE64FF0000901E620
:100BE000BA467EE637467CE67C22002000220020C2
:100BF000A08601000F4B70B51B780C460133DBB2A9
:100C0000012B11D80C4D4FF47A732968A2FB0332E3
:100C100022460E6A01462846B047844204D1074B5B
:100C2000002201201A7070BD4FF4FA7001F0CEF965
:100C30000020F8E710220020B0260020B423002076
:100C4000002307B5024601210DF107008DF807309A
:100C5000FFF7D0FF20B19DF8070003B05DF804FB5B
:100C60004FF0FF30F9E700000A46042108B5FFF70E
:100C7000C1FF80F00100C0B2404208BD30B4054C55
:100C80000A46014623682046DD69034BAC4630BC6A
:100C9000604700BFB0260020A086010070B5104C50
:100CA0000025104E01F0ACFC208030682388834280
:100CB0000CD800252088013801F09EFC23880544CB
:100CC000013BB5F5802F2380F4D370BD01F094FC77
:100CD000336805440133B5F5003F3360E5D3E8E7F9
:100CE000B62300208823002001F058BD00F10060E9
:100CF00000F500300068704700F10060920000F5D8
:100D0000003001F0D9BC0000054B1A68054B1B8868
:100D10009B1A834202D9104401F06EBC0020704738
:100D200088230020B623002038B50446074D29B19A
:100D300028682044BDE8384001F076BC286820448B
:100D400001F060FC0028F3D038BD00BF88230020EC
:100D50000020704700F1FF5000F58F10D0F8000818
:100D600070470000064991F8243033B1002308226F
:100D7000086A81F82430FFF7BFBF0120704700BF29
:100D80008C230020014B1868704700BF0010005CE6
:100D9000194B01380322084470B51D68174BC5F381
:100DA0000B042D0C1E88A6420BD15C680A46013C40
:100DB000824213460FD214F9016F4EB102F8016B53
:100DC000F6E7013A03F10803ECD181420B4602D267
:100DD0002C2203F8012B0424094A1688AE4204D1C0
:100DE000984284BF967803F8016B013C02F104023B
:100DF000F3D1581A70BD00BF0010005C142200200F
:100E0000C8400008022804D1054B4FF400429A6103
:100E100070470128FCD1034B4FF40062F7E700BF95
:100E200000040258000C0258022804D1054B4FF070
:100E300000429A6170470128FCD1034B4FF00062D9
:100E4000F7E700BF00040258000C0258022805D141
:100E5000064A536983F40043536170470128FCD16B
:100E6000034A536983F40063F6E700BF00040258A5
:100E7000000C025870B504464FF47A764CB1412C00
:100E8000254628BF412506FB05F0641B01F09EF8AE
:100E9000F4E770BD002310B5934203D0CC5CC4547A
:100EA0000133F9E710BD0000013810B510F9013F1A
:100EB0003BB191F900409C4203D11AB10131013A92
:100EC000F4E71AB191F90020981A10BD1046FCE71A
:100ED00003460246D01A12F9011B0029FAD17047C5
:100EE00002440346934202D003F8011BFAE770471D
:100EF0002DE9F8431F4D14460746884695F82420EF
:100F000052BBDFF870909CB395F824302BB92022A7
:100F1000FF2148462F62FFF7E3FF95F82400414682
:100F2000C0F1080205EB8000A24228BF2246D6B2DB
:100F30009200FFF7AFFF95F82430A41B17441E441E
:100F40009044E4B2F6B2082E85F82460DBD1FFF7B6
:100F500009FF0028D7D108E02B6A03EB8203834204
:100F6000CFD0FFF7FFFE0028CBD10020BDE8F883EB
:100F70000120FBE78C230020024B1A78024B1A70E9
:100F8000704700BFB42300201022002010B5114C80
:100F9000114800F06FFB21460F4800F097FB2468D2
:100FA0004FF47A70D4F89020D2F8043843F002035A
:100FB000C2F80438FFF75EFF0849204600F094FCB1
:100FC000D4F89020D2F8043823F00203C2F8043891
:100FD00010BD00BF84420008B02600208C420008EB
:100FE00070470000F0B5A1B071B6002301200024C5
:100FF00080261A46194600F04BFA4FF4D067214A72
:101000003D25136923BBD2F810310BBB036804F1F3
:10101000006199600368C3F80CD003685E600368E0
:101020001F6001680B6843F001030B6001680B68E7
:1010300023F01E030B6001680B68DB07FCD4037B05
:101040008034416805FA03F3B4F5001F0B60D8D172
:1010500000F05EFAB4F5001F11D000240A4E0B4DCB
:10106000012001F09BFB3388A34205D92868204466
:10107000013401F0D9FAF6E7002001F08FFB61B6E8
:1010800021B0F0BD00200052B623002088230020AC
:1010900030B50A44084D91420DD011F8013B58403B
:1010A000082340F30004013B2C4013F0FF0384EAC3
:1010B0005000F6D1EFE730BD2083B8ED08B5074BFF
:1010C000074A196801F03D01996053680BB19068B7
:1010D0009847BDE8084001F023BC00BF0000024073
:1010E000B823002008B5084B1968890901F03D01B3
:1010F0008A019A60054AD3680BB110699847BDE828
:10110000084001F00DBC00BF00000240B8230020E1
:1011100008B5084B1968090C01F03D010A049A60F2
:10112000054A53690BB190699847BDE8084001F042
:10113000F7BB00BF00000240B823002008B5084BF1
:101140001968890D01F03D018A059A60054AD36945
:101150000BB1106A9847BDE8084001F0E1BB00BF41
:1011600000000240B823002008B5074B074A596821
:1011700001F03D01D960536A0BB1906A9847BDE810
:10118000084001F0CDBB00BF00000240B8230020A2
:1011900008B5084B5968890901F03D018A01DA60F8
:1011A000054AD36A0BB1106B9847BDE8084001F0BF
:1011B000B7BB00BF00000240B823002008B5084BB1
:1011C0005968090C01F03D010A04DA60054A536BC5
:1011D0000BB1906B9847BDE8084001F0A1BB00BF80
:1011E00000000240B823002008B5084B5968890D5B
:1011F00001F03D018A05DA60054AD36B0BB1106C32
:101200009847BDE8084001F08BBB00BF00000240DA
:10121000B823002008B5074B074A196801F03D01C3
:101220009960536C0BB1906C9847BDE8084001F091
:1012300077BB00BF00040240B823002008B5084B6C
:101240001968890901F03D018A019A60054AD36C49
:101250000BB1106D9847BDE8084001F061BB00BFBD
:1012600000040240B823002008B5084B1968090C97
:1012700001F03D010A049A60054A536D0BB1906D6F
:101280009847BDE8084001F04BBB00BF0004024096
:10129000B823002008B5084B1968890D01F03D01FD
:1012A0008A059A60054AD36D0BB1106E9847BDE868
:1012B000084001F035BB00BF00040240B823002005
:1012C00008B5074B074A596801F03D01D960536ED4
:1012D0000BB1906E9847BDE8084001F021BB00BFFC
:1012E00000040240B823002008B5084B596889095A
:1012F00001F03D018A01DA60054AD36E0BB1106F2F
:101300009847BDE8084001F00BBB00BF0004024055
:10131000B823002008B5084B5968090C01F03D01BD
:101320000A04DA60054A536F0BB1906F9847BDE825
:10133000084001F0F5BA00BF00040240B8230020C5
:1013400008B5084B5968890D01F03D018A05DA603E
:10135000054AD36F13B1D2F880009847BDE8084022
:1013600001F0DEBA00040240B823002000230C493B
:1013700010B51A460B4C0B6054F82300026001EBC9
:10138000430004334260402BF6D1074A4FF0FF334D
:101390009360D360C2F80834C2F80C3410BD00BFAB
:1013A000B8230020D8400008000002400F28F8B5FC
:1013B00010D9102810D0112811D0122808D10F24CC
:1013C0000720DFF8C8E00126DEF80050A04208D967
:1013D000002653E00446F4E70F240020F1E7072439
:1013E000FBE706FA00F73D424AD1264C4FEA001CC3
:1013F0003D4304EB00160EEBC000CEF80050C0E9F0
:101400000123FBB273B12048D0F8D83043F0010378
:10141000C0F8D830D0F8003143F00103C0F80031F3
:10142000D0F8003117F47F4F0ED01748D0F8D830DD
:1014300043F00203C0F8D830D0F8003143F0020383
:10144000C0F80031D0F8003154F80C00036823F0E4
:101450001F030360056815F00105FBD104EB0C03C5
:101460003D2493F80CC05F6804FA0CF43C6021241E
:101470000560446112B1987B00F054F83046F8BD25
:101480000130A3E7D840000800440258B8230020E8
:1014900010B5302484F31188FFF788FF002383F30D
:1014A000118810BD10B50446807B00F051F801236F
:1014B0001549627B03FA02F20B6823EA0203DAB2EF
:1014C0000B6072B9114AD2F8D81021F00101C2F8AC
:1014D000D810D2F8001121F00101C2F80011D2F8A1
:1014E000002113F47F4F0ED1084BD3F8D82022F0FF
:1014F0000202C3F8D820D3F8002122F00202C3F878
:101500000021D3F8003110BDB82300200044025858
:1015100008B5302383F31188FFF7C4FF002383F35A
:10152000118808BD090100F16043012203F5614300
:10153000C9B283F8001300F01F039A4043099B00CF
:1015400003F1604303F56143C3F880211A607047DB
:1015500000F01F0301229A40430900F160409B0004
:1015600000F5614003F1604303F56143C3F8802057
:10157000C3F88021002380F8003370470268436875
:101580001143016003B118477047000013B5406B69
:1015900000F58054D4F8A4381A681178042914D1BD
:1015A000017C022911D11979012312898B40134240
:1015B0000BD101A94C3002F0A3F8D4F8A44802469C
:1015C000019B2179206800F0DFF902B010BD000016
:1015D000143002F025B800004FF0FF33143002F051
:1015E0001FB800004C3002F0F7B800004FF0FF3396
:1015F0004C3002F0F1B80000143001F0F3BF0000ED
:101600004FF0FF31143001F0EDBF00004C3002F01C
:10161000C3B800004FF0FF324C3002F0BDB80000FC
:101620000020704710B500F58054D4F8A4381A682B
:101630001178042917D1017C022914D15979012389
:1016400052898B4013420ED1143001F085FF0246BF
:1016500048B1D4F8A4484FF4407361792068BDE8DC
:10166000104000F07FB910BD406BFFF7DBBF0000FA
:10167000704700007FB5124B012504260446036025
:101680000023057400F1840243602946C0E9023357
:101690000C4B0290143001934FF44073009601F00C
:1016A00037FF094B04F69442294604F14C0002949A
:1016B000CDE900634FF4407301F0FEFF04B070BD4C
:1016C000D8410008691600088D1500080A68302303
:1016D00083F311880B790B3342F823004B791333D2
:1016E00042F823008B7913B10B3342F8230000F545
:1016F0008053C3F8A41802230374002080F31188D8
:101700007047000038B5037F044613B190F8543099
:10171000ABB90125201D0221FFF730FF04F11400B1
:101720006FF00101257700F079FC04F14C0084F89A
:1017300054506FF00101BDE8384000F06FBC38BD77
:1017400010B5012104460430FFF718FF002323776A
:1017500084F8543010BD000038B50446002514301C
:1017600001F0EEFE04F14C00257701F0BDFF201DD5
:1017700084F854500121FFF701FF2046BDE83840AE
:10178000FFF750BF90F8803003F06003202B06D1A4
:1017900090F881200023212A03D81F2A06D8002090
:1017A0007047222AFBD1C0E91D3303E0034A426798
:1017B00007228267C3670120704700BF2C220020E8
:1017C00037B500F58055D5F8A4381A681178042982
:1017D0001AD1017C022917D11979012312898B4072
:1017E000134211D100F14C04204602F03DF858B1EB
:1017F00001A9204601F084FFD5F8A4480246019BC8
:101800002179206800F0C0F803B030BD01F10B036E
:10181000F0B550F8236085B004460D46FEB1302384
:1018200083F3118804EB8507301D0821FFF7A6FE1E
:10183000FB6806F14C005B691B681BB1019001F06D
:101840006DFF019803A901F05BFF024648B1039BBD
:101850002946204600F098F8002383F3118805B04C
:10186000F0BDFB685A691268002AF5D01B8A013B5B
:101870001340F1D104F18002EAE70000133138B5DA
:1018800050F82140ECB1302383F3118804F58053E4
:10189000D3F8A4281368527903EB8203DB689B69B1
:1018A0005D6845B104216018FFF768FE294604F120
:1018B000140001F05BFE2046FFF7B4FE002383F323
:1018C000118838BD7047000001F028B9012340227B
:1018D000002110B5044600F8303BFFF701FB002360
:1018E000C4E9013310BD000010B53023044683F372
:1018F00011882422416000210C30FFF7F1FA2046C4
:1019000001F02EF902230020237080F3118810BD0E
:1019100070B500EB8103054650690E461446DA6047
:1019200018B110220021FFF7DBFAA06918B11022CC
:101930000021FFF7D5FA31462846BDE8704001F096
:1019400015BA000083682022002103F0011310B5AE
:10195000044683601030FFF7C3FA2046BDE810400C
:1019600001F090BAF0B4012500EB810447898D4065
:10197000E4683D43A469458123600023A26063605D
:10198000F0BC01F0ADBA0000F0B4012500EB810419
:1019900007898D40E4683D43646905812360002325
:1019A000A2606360F0BC01F023BB000070B50223AD
:1019B00000250446242203702946C0F888500C30C4
:1019C00040F8045CFFF78CFA204684F8705001F070
:1019D00061F963681B6823B129462046BDE8704061
:1019E000184770BD0378052B10B504460AD080F85F
:1019F0008C300523037043681B680BB104219847A2
:101A00000023A36010BD00000178052906D190F8DD
:101A10008C20436802701B6803B1184770470000B0
:101A200070B590F87030044613B1002380F8703020
:101A300004F18002204601F049FA63689B68B3B95B
:101A400094F8803013F0600535D00021204601F075
:101A50003BFD0021204601F02BFD63681B6813B19C
:101A6000062120469847062384F8703070BD204632
:101A700098470028E4D0B4F88630A26F9A4288BF15
:101A8000A36794F98030A56F002B4FF0300380F2EC
:101A90000381002D00F0F280092284F8702083F386
:101AA000118800212046D4E91D23FFF76DFF002394
:101AB00083F31188DAE794F8812003F07F0343EA87
:101AC000022340F20232934200F0C58021D8B3F5E0
:101AD000807F48D00DD8012B3FD0022B00F093809F
:101AE000002BB2D104F1880262670222A267E36789
:101AF000C1E7B3F5817F00F09B80B3F5407FA4D1AF
:101B000094F88230012BA0D1B4F8883043F002035E
:101B100032E0B3F5006F4DD017D8B3F5A06F31D0D8
:101B2000A3F5C063012B90D86368204694F8822007
:101B30005E6894F88310B4F88430B047002884D0ED
:101B4000436863670368A3671AE0B3F5106F36D084
:101B500040F6024293427FF478AF5C4B6367022306
:101B6000A3670023C3E794F88230012B7FF46DAFA5
:101B7000B4F8883023F00203A4F88830C4E91D5576
:101B8000E56778E7B4F88030B3F5A06F0ED194F82C
:101B90008230204684F88A3001F0DAF863681B68E6
:101BA00013B1012120469847032323700023C4E981
:101BB0001D339CE704F18B0363670123C3E723789C
:101BC000042B10D1302383F311882046FFF7BAFE8F
:101BD00085F311880321636884F88B5021701B689A
:101BE0000BB12046984794F88230002BDED084F861
:101BF0008B300423237063681B68002BD6D002212E
:101C000020469847D2E794F8843020461D0603F01A
:101C10000F010AD501F04CF9012804D002287FF405
:101C200014AF2B4B9AE72B4B98E701F033F9F3E70E
:101C300094F88230002B7FF408AF94F8843013F0CE
:101C40000F01B3D01A06204602D501F055FCADE7CE
:101C500001F046FCAAE794F88230002B7FF4F5AE41
:101C600094F8843013F00F01A0D01B06204602D553
:101C700001F02AFC9AE701F01BFC97E7142284F894
:101C8000702083F311882B462A4629462046FFF709
:101C900069FE85F31188E9E65DB1152284F87020AC
:101CA00083F3118800212046D4E91D23FFF75AFE53
:101CB000FDE60B2284F8702083F311882B462A4618
:101CC00029462046FFF760FEE3E700BF0842000810
:101CD000004200080442000838B590F8703004460D
:101CE000002B3ED0063BDAB20F2A34D80F2B32D865
:101CF000DFE803F03731310822323131313131310F
:101D000031313737856FB0F886309D4214D2C368C1
:101D10001B8AB5FBF3F203FB12556DB9302383F335
:101D200011882B462A462946FFF72EFE85F3118897
:101D30000A2384F870300EE0142384F870303023C6
:101D400083F31188002320461A461946FFF70AFE3E
:101D5000002383F3118838BDC36F03B19847002374
:101D6000E7E70021204601F0AFFB0021204601F00B
:101D70009FFB63681B6813B1062120469847062322
:101D8000D7E7000010B590F870300446142B29D026
:101D900017D8062B05D001D81BB110BD093B022B6B
:101DA000FBD80021204601F08FFB0021204601F0E6
:101DB0007FFB63681B6813B1062120469847062302
:101DC00019E0152BE9D10B2380F87030302383F311
:101DD000118800231A461946FFF7D6FD002383F326
:101DE0001188DAE7C3689B695B68002BD5D1C36FA4
:101DF00003B19847002384F87030CEE7002382684F
:101E0000037503691B6899689142FBD25A680360A5
:101E10004260106058607047002382680375036950
:101E20001B6899689142FBD85A6803604260106051
:101E30005860704708B50846302383F311880B7D3E
:101E4000032B05D0042B0DD02BB983F3118808BDCB
:101E50008B6900221A604FF0FF338361FFF7CEFFDA
:101E60000023F2E7D1E9003213605A60F3E7000083
:101E7000FFF7C4BF054BD96808751868026853603E
:101E80001A600122D8600275FEF7BCBA4024002017
:101E90000C4B30B5DD684B1C87B004460FD02B4689
:101EA000094A684600F04EF92046FFF7E3FF009B21
:101EB00013B1684600F050F9A86907B030BDFFF7CC
:101EC000D9FFF9E740240020351E0008044B1A68AA
:101ED000DB6890689B68984294BF0020012070479F
:101EE00040240020084B10B51C68D8682268536055
:101EF0001A600122DC602275FFF78EFF0146204642
:101F0000BDE81040FEF77EBA4024002038B5074CEB
:101F100001230025064907482370656001F0E2FCB3
:101F20000223237085F3118838BD00BFA826002046
:101F3000104200084024002000F044B9034A5168D0
:101F400053685B1A9842FBD8704700BF001000E04E
:101F50008B600223086108468B8270478368A3F177
:101F6000840243F8142C026943F8442C426943F874
:101F7000402C094A43F8242CC268A3F1200043F8FE
:101F8000182C022203F80C2C002203F80B2C034A15
:101F900043F8102C704700BF1D04000840240020A7
:101FA00008B5FFF7DBFFBDE80840FFF761BF0000A1
:101FB000024BDB6898610F20FFF75CBF40240020D4
:101FC000302383F31188FFF7F3BF000008B5014603
:101FD000302383F311880820FFF75AFF002383F38F
:101FE000118808BD064BDB6839B1426818605A6039
:101FF000136043600420FFF74BBF4FF0FF30704782
:10200000402400200368984206D01A68026050609D
:1020100018469961FFF72CBF7047000038B5044699
:102020000D462068844200D138BD036823605C609F
:102030008561FFF71DFFF4E7036810B59C68A242B5
:102040000CD85C688A600B604C60216059609968AC
:102050008A1A9A604FF0FF33836010BD121B1B6811
:10206000ECE700000A2938BF0A2170B504460D4686
:102070000A26601901F02EFC01F016FC041BA54293
:1020800003D8751C04462E46F3E70A2E04D9012016
:10209000BDE8704001F066BC70BD0000F8B5144B9F
:1020A0000D460A2A4FF00A07D96103F11001826038
:1020B00038BF0A22416019691446016048601861FE
:1020C000A81801F0F7FB01F0EFFB431B0646A34203
:1020D00006D37C1C28192746354601F0FBFBF2E7A6
:1020E0000A2F04D90120BDE8F84001F03BBCF8BD3F
:1020F00040240020F8B506460D4601F0D5FB0F4AF6
:10210000134653F8107F9F4206D12A4601463046B7
:10211000BDE8F840FFF7C2BFD169BB68441A2C196B
:1021200028BF2C46A34202D92946FFF79BFF22462F
:1021300031460348BDE8F840FFF77EBF4024002049
:1021400050240020C0E90323002310B45DF8044BA1
:102150004361FFF7CFBF000010B5194C23699842C7
:102160000DD08168D0E9003213605A609A680A4441
:102170009A60002303604FF0FF33A36110BD026833
:10218000234643F8102F53600022026022699A42CE
:1021900003D1BDE8104001F097BB936881680B4400
:1021A000936001F081FB2269E1699268441AA242BE
:1021B000E4D91144BDE81040091AFFF753BF00BF2E
:1021C000402400202DE9F047DFF8BC8008F110071B
:1021D0002C4ED8F8105001F067FBD8F81C40AA68C4
:1021E000031B9A423ED814444FF00009D5E900324F
:1021F000C8F81C4013605A60C5F80090D8F8103039
:10220000B34201D101F060FB89F31188D5E90331B4
:1022100028469847302383F311886B69002BD8D068
:1022200001F042FB6A69A0EB040982464A450DD2DF
:10223000022001F097FB0022D8F81030B34208D1F9
:1022400051462846BDE8F047FFF728BF121A22443E
:10225000F2E712EB09092946384638BF4A46FFF72C
:10226000EBFEB5E7D8F81030B34208D01444C8F8F4
:102270001C00211AA960BDE8F047FFF7F3BEBDE8D6
:10228000F08700BF50240020402400200020704729
:10229000FEE70000704700004FF0FF30704700007D
:1022A00002290CD0032904D00129074818BF0020B7
:1022B0007047032A05D8054800EBC2007047044860
:1022C00070470020704700BFE84200083C22002011
:1022D0009C42000870B59AB005460846144601A90C
:1022E00000F0C2F801A8FEF7F3FD431C0022C6B2BD
:1022F0005B001046C5E9003423700323023404F860
:10230000013C01ABD1B202348E4201D81AB070BD8B
:1023100013F8011B013204F8010C04F8021CF1E768
:1023200008B5302383F311880348FFF749FA0023E7
:1023300083F3118808BD00BFB026002090F88030DC
:1023400003F01F02012A07D190F881200B2A03D144
:102350000023C0E91D3315E003F06003202B08D1F2
:10236000B0F884302BB990F88120212A03D81F2A95
:1023700004D8FFF707BA222AEBD0FAE7034A4267EC
:1023800007228267C3670120704700BF3322002005
:1023900007B5052917D8DFE801F019160319192028
:1023A000302383F31188104A01210190FFF7B0FA1E
:1023B000019802210D4AFFF7ABFA0D48FFF7CCF95F
:1023C000002383F3118803B05DF804FB302383F30B
:1023D00011880748FFF796F9F2E7302383F3118855
:1023E0000348FFF7ADF9EBE73C4200086042000804
:1023F000B026002038B50C4D0C4C2A460C4904F18F
:102400000800FFF767FF05F1CA0204F1100009494F
:10241000FFF760FF05F5CA7204F118000649BDE830
:102420003840FFF757BF00BF883F00203C22002004
:102430001C420008264200083142000870B50446DC
:1024400008460D46FEF744FDC6B220460134037827
:102450000BB9184670BD32462946FEF725FD002807
:10246000F3D10120F6E700002DE9F84F05460C46B0
:10247000FEF72EFD2A49C6B22846FFF7DFFF08B156
:102480000136F6B227492846FFF7D8FF08B11036C3
:10249000F6B2632E0DD8DFF88890DFF888A0224FBF
:1024A000DFF88CB0DFF88C802E7846B92670BDE856
:1024B000F88F29462046BDE8F84F01F0E7BD252EEC
:1024C0002AD1072249462846FEF7EEFC50B9D8F833
:1024D00000300735083444F8083CD8F8043044F894
:1024E000043CE1E7082251462846FEF7DDFC98B996
:1024F000A21C0E4B197802320909C95D02F8041CAE
:1025000013F8011B01F00F015B45C95D02F8031CC4
:10251000F0D118340835C7E7013504F8016BC3E77B
:1025200008430008314200081943000800E8F11F81
:102530000CE8F11F10430008BFF34F8F044B1A69DA
:102540005107FCD1D3F810215207F8D1704700BFD2
:102550000020005208B50D4B1B78ABB9FFF7ECFF1C
:102560000B4BDA68D10704D50A4A5A6002F1883267
:102570005A60D3F80C21D20706D5064AC3F80421C5
:1025800002F18832C3F8042108BD00BFE6410020F3
:10259000002000522301674508B5114B1B78F3B9A1
:1025A000104B1A69510703D5DA6842F04002DA602D
:1025B000D3F81021520705D5D3F80C2142F0400280
:1025C000C3F80C21FFF7B8FF064BDA6842F00102AE
:1025D000DA60D3F80C2142F00102C3F80C2108BDE7
:1025E000E6410020002000520F289ABF00F58060CD
:1025F00040040020704700004FF400307047000096
:10260000102070470F2808B50BD8FFF7EDFF00F535
:1026100000330268013204D104308342F9D1012031
:1026200008BD0020FCE700000F2838B505463FD85C
:10263000FFF782FF1F4CFFF78DFF4FF0FF33072896
:102640006361C4F814311DD82361FFF775FF0302DD
:1026500043F02403E360E36843F08003E36023690D
:102660005A07FCD42846FFF767FFFFF7BDFF4FF47A
:10267000003100F0F5F82846FFF78EFFBDE838403E
:10268000FFF7C0BFC4F81031FFF756FFA0F10803F1
:102690001B0243F02403C4F80C31D4F80C3143F08E
:1026A0008003C4F80C31D4F810315B07FBD4D9E7B0
:1026B000002038BD002000522DE9F84F05460C4699
:1026C000104645EA0203DE0602D00020BDE8F88F7E
:1026D00020F01F00DFF8BCB0DFF8BCA0FFF73AFF26
:1026E00004EB0008444503D10120FFF755FFEDE757
:1026F00020222946204601F0B9FC10B920352034AB
:10270000F0E72B4605F120021F68791CDDD1043368
:102710009A42F9D105F178431B481C4EB3F5801F4E
:102720001B4B38BF184603F1F80332BFD946D146D8
:102730001E46FFF701FF0760A5EB040C336804F1A8
:102740001C0143F002033360231FD9F8007017F017
:102750000507FAD153F8042F8B424CF80320F4D12B
:10276000BFF34F8FFFF7E8FE4FF0FF3320222146E3
:1027700003602846336823F00203336001F076FCDF
:102780000028BBD03846B0E7142100520C2000527C
:1027900014200052102000521021005210B5084C95
:1027A000237828B11BB9FFF7D5FE0123237010BD94
:1027B000002BFCD02070BDE81040FFF7EDBE00BF3D
:1027C000E64100200244074BD2B210B5904200D13E
:1027D00010BD441C00B253F8200041F8040BE0B2D5
:1027E000F4E700BF504000580E4B30B51C6F240476
:1027F00005D41C6F1C671C6F44F400441C670A4C12
:1028000002442368D2B243F480732360074B9042A2
:1028100000D130BD441C51F8045B00B243F8205095
:10282000E0B2F4E700440258004802585040005813
:1028300007B5012201A90020FFF7C4FF019803B0EA
:102840005DF804FB13B50446FFF7F2FFA04205D084
:10285000012201A900200194FFF7C6FF02B010BDBC
:102860000144BFF34F8F064B884204D3BFF34F8F11
:10287000BFF36F8F7047C3F85C022030F4E700BFEE
:1028800000ED00E0034B1A681AB9034AD2F8D024CD
:102890001A607047E84100200040025808B5FFF771
:1028A000F1FF024B1868C0F3806008BDE8410020CA
:1028B000EFF30983054968334A6B22F001024A634A
:1028C00083F30988002383F31188704700EF00E049
:1028D000302080F3118862B60D4B0E4AD96821F47E
:1028E000E0610904090C0A430B49DA60D3F8FC20C3
:1028F00042F08072C3F8FC20084AC2F8B01F116889
:1029000041F0010111602022DA7783F8220070473C
:1029100000ED00E00003FA0555CEACC5001000E064
:10292000302310B583F311880E4B5B6813F40063FA
:1029300014D0F1EE103AEFF309844FF08073683C45
:10294000E361094BDB6B236684F30988FFF7BEFA6A
:1029500010B1064BA36110BD054BFBE783F3118853
:10296000F9E700BF00ED00E000EF00E02F040008F1
:102970003204000870B5BFF34F8FBFF36F8F1A4A50
:102980000021C2F85012BFF34F8FBFF36F8F53690E
:1029900043F400335361BFF34F8FBFF36F8FC2F81F
:1029A0008410BFF34F8FD2F8803043F6E074C3F346
:1029B000C900C3F34E335B0103EA0406014646EA4D
:1029C00081750139C2F86052F9D2203B13F1200F12
:1029D000F2D1BFF34F8F536943F480335361BFF398
:1029E0004F8FBFF36F8F70BD00ED00E0FEE700007A
:1029F000214B2248224A70B5904237D3214BC11E49
:102A0000DA1C121A22F003028B4238BF0022002186
:102A1000FEF766FA1C4A0023C2F88430BFF34F8FDA
:102A2000D2F8803043F6E074C3F3C900C3F34E33E9
:102A30005B0103EA0406014646EA81750139C2F8E2
:102A40006C52F9D2203B13F1200FF2D1BFF34F8F1C
:102A5000BFF36F8FBFF34F8FBFF36F8F0023C2F8A9
:102A60005032BFF34F8FBFF36F8F70BD53F8041B0D
:102A700040F8041BC0E700BF04450008BC43002029
:102A8000BC430020BC43002000ED00E0074BD3F81E
:102A9000D81021EA0001C3F8D810D3F8002122EAA7
:102AA0000002C3F80021D3F80031704700440258F7
:102AB00070B5D0E9244300224FF0FF359E6804EB47
:102AC00042135101D3F80009002805DAD3F80009B0
:102AD00040F08040C3F80009D3F8000B002805DA65
:102AE000D3F8000B40F08040C3F8000B01326318AC
:102AF0009642C3F80859C3F8085BE0D24FF00113BF
:102B0000C4F81C3870BD0000890141F0200101614A
:102B100003699B06FCD41220FFF710BA10B50A4CCB
:102B20002046FEF7D3FE094BC4F89030084BC4F89A
:102B30009430084C2046FEF7C9FE074BC4F890308D
:102B4000064BC4F8943010BDEC4100200000084052
:102B50005043000888420020000004405C43000805
:102B600070B503780546012B5CD1434BD0F89040FB
:102B7000984258D1414B0E216520D3F8D82042F01D
:102B80000062C3F8D820D3F8002142F00062C3F8F5
:102B90000021D3F80021D3F8802042F00062C3F86E
:102BA0008020D3F8802022F00062C3F88020D3F880
:102BB0008030FEF7B7FC324BE360324BC4F800388C
:102BC0000023D5F89060C4F8003EC02323604FF482
:102BD0000413A3633369002BFCDA01230C20336157
:102BE000FFF7ACF93369DB07FCD41220FFF7A6F935
:102BF0003369002BFCDA00262846A660FFF758FF51
:102C00006B68C4F81068DB68C4F81468C4F81C6802
:102C100083BB1D4BA3614FF0FF336361A36843F097
:102C20000103A36070BD194B9842C9D1134B4FF0FB
:102C30008060D3F8D82042F00072C3F8D820D3F8CF
:102C4000002142F00072C3F80021D3F80021D3F82C
:102C5000802042F00072C3F88020D3F8802022F058
:102C60000072C3F88020D3F88030FFF70FFF0E21E9
:102C70004D209EE7064BCDE7EC4100200044025872
:102C80004014004003002002003C30C08842002075
:102C9000083C30C0F8B5D0F89040054600214FF010
:102CA00000662046FFF730FFD5F8941000234FF060
:102CB00001128F684FF0FF30C4F83438C4F81C2874
:102CC00004EB431201339F42C2F80069C2F8006B63
:102CD000C2F80809C2F8080BF2D20B68D5F89020A8
:102CE000C5F89830636210231361166916F0100658
:102CF000FBD11220FFF722F9D4F8003823F4FE6349
:102D0000C4F80038A36943F4402343F01003A361DF
:102D10000923C4F81038C4F814380B4BEB604FF09B
:102D2000C043C4F8103B094BC4F8003BC4F8106919
:102D3000C4F80039D5F8983003F1100243F4801339
:102D4000C5F89820A362F8BD2C430008408000100D
:102D5000D0F8902090F88A10D2F8003823F4FE635F
:102D600043EA0113C2F80038704700002DE9F84328
:102D700000EB8103D0F890500C468046DA680FFAD9
:102D800081F94801166806F00306731E022B05EB55
:102D900041134FF0000194BFB604384EC3F8101B26
:102DA0004FF0010104F1100398BF06F1805601FABB
:102DB00003F3916998BF06F5004600293AD0578A77
:102DC00004F15801374349016F50D5F81C180B43E3
:102DD0000021C5F81C382B180127C3F81019A7408B
:102DE0005369611E9BB3138A928B9B08012A88BF8B
:102DF0005343D8F89820981842EA034301F140025F
:102E00002146C8F89800284605EB82025360FFF778
:102E10007BFE08EB8900C3681B8A43EA845348346D
:102E20001E4364012E51D5F81C381F43C5F81C7889
:102E3000BDE8F88305EB4917D7F8001B21F40041E2
:102E4000C7F8001BD5F81C1821EA0303C0E704F1FA
:102E50003F030B4A2846214605EB83035A60FFF7E0
:102E600053FE05EB4910D0F8003923F40043C0F8B5
:102E70000039D5F81C3823EA0707D7E7008000108F
:102E800000040002D0F894201268C0F89820FFF7E0
:102E90000FBE00005831D0F8903049015B5813F450
:102EA000004004D013F4001F0CBF02200120704723
:102EB0004831D0F8903049015B5813F4004004D0F9
:102EC00013F4001F0CBF02200120704700EB8101AA
:102ED000CB68196A0B6813604B6853607047000039
:102EE00000EB810330B5DD68AA691368D36019B9B6
:102EF000402B84BF402313606B8A1468D0F8902065
:102F00001C4402EB4110013C09B2B4FBF3F46343EF
:102F1000033323F0030343EAC44343F0C043C0F840
:102F2000103B2B6803F00303012B0ED1D2F80838B5
:102F300002EB411013F4807FD0F8003B14BF43F044
:102F4000805343F00053C0F8003B02EB4112D2F82B
:102F5000003B43F00443C2F8003B30BD2DE9F04193
:102F6000D0F8906005460C4606EB4113D3F8087B79
:102F70003A07C3F8087B08D5D6F814381B0704D5E0
:102F800000EB8103DB685B689847FA071FD5D6F82A
:102F90001438DB071BD505EB8403D968CCB98B69E2
:102FA000488A5A68B2FBF0F600FB16228AB9186804
:102FB000DA6890420DD2121AC3E90024302383F359
:102FC000118821462846FFF78BFF84F31188BDE85E
:102FD000F081012303FA04F26B8923EA02036B8177
:102FE000CB68002BF3D021462846BDE8F0411847B6
:102FF00000EB81034A0170B5DD68D0F890306C6950
:103000002668E66056BB1A444FF40020C2F8100947
:103010002A6802F00302012A0AB20ED1D3F8080886
:1030200003EB421410F4807FD4F8000914BF40F081
:10303000805040F00050C4F8000903EB4212D2F86F
:10304000000940F00440C2F800090122D3F8340816
:1030500002FA01F10143C3F8341870BD19B9402ECA
:1030600084BF4020206020681A442E8A8419013CC5
:10307000B4FBF6F440EAC44040F00050C6E700005C
:103080002DE9F843D0F8906005460C464F0106EB59
:103090004113D3F8088918F0010FC3F808891CD030
:1030A000D6F81038DB0718D500EB8103D3F80CC035
:1030B000DCF81430D3F800E0DA68964530D2A2EBA1
:1030C0000E024FF000091A60C3F80490302383F316
:1030D0001188FFF78DFF89F3118818F0800F1DD03C
:1030E000D6F834380126A640334217D005EB8403C6
:1030F0000134D5F89050D3F80CC0E4B22F44DCF87A
:10310000142005EB0434D2F800E05168714514D363
:10311000D5F8343823EA0606C5F83468BDE8F883E4
:10312000012303FA01F2038923EA02030381DCF895
:103130000830002BD1D09847CFE7AEEB0103BCF8A5
:103140001000834228BF0346D7F8180980B2B3EBBA
:10315000800FE3D89068A0F1040959F8048FC4F8EF
:103160000080A0EB09089844B8F1040FF5D8184482
:103170000B4490605360C8E72DE9F84FD0F89050A9
:1031800004466E69AB691E4016F480586E6103D028
:10319000BDE8F84FFEF70ABC002E12DAD5F8003E63
:1031A0009B0705D0D5F8003E23F00303C5F8003E89
:1031B000D5F80438204623F00103C5F80438FEF79B
:1031C00023FC370505D52046FFF772FC2046FEF7A5
:1031D00009FCB0040CD5D5F8083813F0060FEB68DD
:1031E00023F470530CBF43F4105343F4A053EB602B
:1031F00031071BD56368DB681BB9AB6923F0080393
:10320000AB612378052B0CD1D5F8003E9A0705D089
:10321000D5F8003E23F00303C5F8003E2046FEF734
:10322000F3FB6368DB680BB120469847F30200F1BB
:10323000BA80B70226D5D4F8909000274FF0010A43
:1032400009EB4712D2F8003B03F44023B3F5802F7B
:1032500011D1D2F8003B002B0DDA62890AFA07F38C
:1032600022EA0303638104EB8703DB68DB6813B1A5
:103270003946204698470137D4F89430FFB29B680E
:103280009F42DDD9F00619D5D4F89000026AC2F346
:103290000A1702F00F0302F4F012B2F5802F00F0CB
:1032A000CA80B2F5402F09D104EB8303002200F558
:1032B0008050DB681B6A974240F0B0803003D5F83D
:1032C000185835D5E90303D500212046FFF746FEFF
:1032D000AA0303D501212046FFF740FE6B0303D567
:1032E00002212046FFF73AFE2F0303D50321204693
:1032F000FFF734FEE80203D504212046FFF72EFE37
:10330000A90203D505212046FFF728FE6A0203D54E
:1033100006212046FFF722FE2B0203D50721204677
:10332000FFF71CFEEF0103D508212046FFF716FE2C
:10333000700340F1A780E90703D500212046FFF77D
:103340009FFEAA0703D501212046FFF799FE6B07D0
:1033500003D502212046FFF793FE2F0703D5032153
:103360002046FFF78DFEEE0603D504212046FFF729
:1033700087FEA80603D505212046FFF781FE6906D2
:1033800003D506212046FFF77BFE2A0603D5072139
:103390002046FFF775FEEB0574D520460821BDE8F1
:1033A000F84FFFF76DBED4F890904FF0000B4FF040
:1033B000010AD4F894305FFA8BF79B689F423FF67E
:1033C00038AF09EB4713D3F8002902F44022B2F5D5
:1033D000802F20D1D3F80029002A1CDAD3F8002945
:1033E00042F09042C3F80029D3F80029002AFBDB01
:1033F0003946D4F89000FFF787FB22890AFA07F3D1
:1034000022EA0303238104EB8703DB689B6813B183
:103410003946204698470BF1010BCAE7910701D1C5
:10342000D0F80080072A02F101029CBF03F8018B4B
:103430004FEA18283FE704EB830300F58050DA6871
:10344000D2F818C0DCF80820DCE9001CA1EB0C0C59
:1034500000218F4208D1DB689B699A683A449A60E0
:103460005A683A445A6029E711F0030F01D1D0F8A5
:1034700000808C4501F1010184BF02F8018B4FEA05
:103480001828E6E7BDE8F88F08B50348FFF774FE93
:10349000BDE80840FFF744BAEC41002008B50348F6
:1034A000FFF76AFEBDE80840FFF73ABA88420020FD
:1034B000D0F8903003EB4111D1F8003B43F40013F6
:1034C000C1F8003B70470000D0F8903003EB411189
:1034D000D1F8003943F40013C1F8003970470000F7
:1034E000D0F8903003EB4111D1F8003B23F40013E6
:1034F000C1F8003B70470000D0F8903003EB411159
:10350000D1F8003923F40013C1F8003970470000E6
:1035100030B50433039C0172002104FB0325C16014
:10352000C0E90653049B0363059BC0E90000C0E9A2
:103530000422C0E90842C0E90A11436330BD00001B
:103540000022416AC260C0E90411C0E90A226FF09A
:103550000101FEF763BD0000D0E90432934201D1BE
:10356000C2680AB9181D70470020704703691960C6
:103570000021C2680132C260C26913448269934269
:10358000036124BF436A0361FEF73CBD38B50446BE
:103590000D46E3683BB162690020131D1268A36207
:1035A0001344E36207E0237A33B929462046FEF745
:1035B00019FD0028EDDA38BD6FF00100FBE70000CF
:1035C000C368C269013BC360436913448269934283
:1035D000436124BF436A436100238362036B03B1E9
:1035E0001847704770B53023044683F31188866A04
:1035F0003EB9FFF7CBFF054618B186F31188284680
:1036000070BDA36AE26A13F8015B9342A36202D31E
:103610002046FFF7D5FF002383F31188EFE7000072
:103620002DE9F84F04460E46174698464FF03009EC
:1036300089F311880025AA46D4F828B0BBF1000F01
:1036400009D141462046FFF7A1FF20B18BF3118835
:103650002846BDE8F88FD4E90A12A7EB050B521AE9
:10366000934528BF9346BBF1400F1BD9334601F168
:10367000400251F8040B914243F8040BF9D1A36ABC
:10368000403640354033A362D4E90A239A4202D33C
:103690002046FFF795FF8AF31188BD42D8D289F3FF
:1036A0001188C9E730465A46FDF7F4FBA36A5E4429
:1036B0005D445B44A362E7E710B5029C04330172EA
:1036C00003FB0421C460C0E906130023C0E90A33E8
:1036D000039B0363049BC0E90000C0E90422C0E926
:1036E0000842436310BD0000026A6FF00101C2602E
:1036F000426AC0E904220022C0E90A22FEF78EBC19
:10370000D0E904239A4201D1C26822B9184650F880
:10371000043B0B60704700231846FAE7C36800219A
:10372000C2690133C36043691344826993424361B0
:1037300024BF436A4361FEF765BC000038B5044608
:103740000D46E3683BB1236900201A1DA262E269BD
:103750001344E36207E0237A33B929462046FEF793
:1037600041FC0028EDDA38BD6FF00100FBE70000F6
:1037700003691960C268013AC260C2691344826970
:103780009342036124BF436A036100238362036B96
:1037900003B118477047000070B530230D4604464A
:1037A000114683F31188866A2EB9FFF7C7FF10B15F
:1037B00086F3118870BDA36A1D70A36AE26A0133A3
:1037C0009342A36204D3E16920460439FFF7D0FF96
:1037D000002080F31188EDE72DE9F84F04460D46EF
:1037E000904699464FF0300A8AF311880026B34676
:1037F000A76A4FB949462046FFF7A0FF20B187F3DB
:1038000011883046BDE8F88FD4E90A073A1AA8EBC8
:103810000607974228BF1746402F1BD905F14003E2
:1038200055F8042B9D4240F8042BF9D1A36A403689
:103830004033A362D4E90A239A4204D3E1692046C3
:103840000439FFF795FF8BF311884645D9D28AF3E7
:103850001188CDE729463A46FDF71CFBA36A3D4493
:103860003E443B44A362E5E7D0E904239A4217D1E2
:10387000C3689BB1836A8BB1043B9B1A0ED0136063
:10388000C368013BC360C3691A4483699A420261F9
:1038900024BF436A036100238362012318467047F3
:1038A0000023FBE700F024B9014B586A704700BFC2
:1038B000000C0040034B002258631A610222DA60B8
:1038C000704700BF000C0040014B0022DA607047D7
:1038D000000C0040014B5863704700BF000C0040D3
:1038E000FEE7000070B51B4B0025044686B058600B
:1038F0000E4685620163FEF7EBFF04F11003A5603D
:10390000E562C4E904334FF0FF33C4E90044C4E97D
:103910000635FFF7C9FF2B46024604F13401204665
:10392000C4E9082380230C4A2565FEF711FB012317
:103930000A4AE06000920375684672680192B268B4
:10394000CDE90223064BCDE90435FEF729FB06B08D
:1039500070BD00BFA8260020684300086D43000822
:10396000E1380008024AD36A1843D062704700BFAA
:10397000402400204B6843608B688360CB68C36041
:103980000B6943614B6903628B6943620B68036097
:103990007047000008B53C4B40F2FF713B48D3F83C
:1039A00088200A43C3F88820D3F8882022F4FF62D5
:1039B00022F00702C3F88820D3F88820D3F8E0204B
:1039C0000A43C3F8E020D3F808210A43C3F80821CA
:1039D0002F4AD3F808311146FFF7CCFF00F580607D
:1039E00002F11C01FFF7C6FF00F5806002F138010B
:1039F000FFF7C0FF00F5806002F15401FFF7BAFF46
:103A000000F5806002F17001FFF7B4FF00F58060FF
:103A100002F18C01FFF7AEFF00F5806002F1A80112
:103A2000FFF7A8FF00F5806002F1C401FFF7A2FFD5
:103A300000F5806002F1E001FFF79CFF00F5806077
:103A400002F1FC01FFF796FF02F58C7100F5806032
:103A5000FFF790FF00F018F90E4BD3F8902242F0D8
:103A60000102C3F89022D3F8942242F00102C3F875
:103A700094220522C3F898204FF06052C3F89C208E
:103A8000054AC3F8A02008BD0044025800000258AF
:103A90007443000800ED00E01F00080308B500F0C3
:103AA000C7FAFEF733FA0F4BD3F8DC2042F040029E
:103AB000C3F8DC20D3F8042122F04002C3F804212B
:103AC000D3F80431084B1A6842F008021A601A68E9
:103AD00042F004021A60FEF7D5FEBDE80840FEF78A
:103AE00089BC00BF0044025800180248704700001B
:103AF000114BD3F8E82042F00802C3F8E820D3F8CD
:103B0000102142F00802C3F810210C4AD3F81031FA
:103B1000D36B43F00803D363C722094B9A624FF07B
:103B2000FF32DA6200229A615A63DA605A60012237
:103B30005A611A60704700BF004402580010005CD0
:103B4000000C0040094A08B51169D3680B40D9B28E
:103B50009B076FEA0101116107D5302383F31188B8
:103B6000FEF7EAF9002383F3118808BD000C00403A
:103B7000064BD3F8DC200243C3F8DC20D3F8042141
:103B80001043C3F80401D3F80431704700440258CD
:103B900008B53C4B4FF0FF31D3F8802062F0004273
:103BA000C3F88020D3F8802002F00042C3F88020C0
:103BB000D3F88020D3F88420C3F88410D3F884206D
:103BC0000022C3F88420D3F88400D86F40F0FF406F
:103BD00040F4FF0040F4DF4040F07F00D867D86F2A
:103BE00020F0FF4020F4FF0020F4DF4020F07F00B1
:103BF000D867D86FD3F888006FEA40506FEA50500A
:103C0000C3F88800D3F88800C0F30A00C3F888001E
:103C1000D3F88800D3F89000C3F89010D3F8900040
:103C2000C3F89020D3F89000D3F89400C3F8941010
:103C3000D3F89400C3F89420D3F89400D3F89800F4
:103C4000C3F89810D3F89800C3F89820D3F89800D8
:103C5000D3F88C00C3F88C10D3F88C00C3F88C20F8
:103C6000D3F88C00D3F89C00C3F89C10D3F89C10B8
:103C7000C3F89C20D3F89C30FDF778FBBDE80840E2
:103C800000F0AEB90044025808B50122534BC3F806
:103C90000821534BD3F8F42042F00202C3F8F42079
:103CA000D3F81C2142F00202C3F81C210222D3F8EF
:103CB0001C314C4BDA605A689104FCD54A4A1A60B0
:103CC00001229A60494ADA6000221A614FF44042A8
:103CD0009A61444B9A699204FCD51A6842F4807246
:103CE0001A603F4B1A6F12F4407F04D04FF48032B9
:103CF0001A6700221A671A6842F001021A60384BEC
:103D00001A685007FCD500221A611A6912F03802AD
:103D1000FBD1012119604FF0804159605A67344A44
:103D2000DA62344A1A611A6842F480321A602C4B03
:103D30001A689103FCD51A6842F480521A601A6816
:103D40009204FCD52C4A2D499A6200225A631963C9
:103D500001F57C01DA6301F2E71199635A64284A9C
:103D60001A64284ADA621A6842F0A8521A601C4B98
:103D70001A6802F02852B2F1285FF9D148229A61FC
:103D80004FF48862DA6140221A621F4ADA641F4ADD
:103D90001A651F4A5A651F4A9A6532231E4A1360E4
:103DA000136803F00F03022BFAD10D4A136943F095
:103DB00003031361136903F03803182BFAD14FF092
:103DC0000050FFF7D5FE4FF08040FFF7D1FE4FF0D7
:103DD0000040BDE80840FFF7CBBE00BF00800051A7
:103DE000004402580048025800C000F002000001E0
:103DF0000000FF01008890082220400063020901B2
:103E0000470E0508DD0BBF01200000200000011057
:103E10000910E00000010110002000524FF0B042F4
:103E200008B5D2F8883003F00103C2F8883023B116
:103E3000044A13680BB150689847BDE80840FEF784
:103E40006FBD00BF3C4300204FF0B04208B5D2F830
:103E5000883003F00203C2F8883023B1044A936823
:103E60000BB1D0689847BDE80840FEF759BD00BFC8
:103E70003C4300204FF0B04208B5D2F8883003F040
:103E80000403C2F8883023B1044A13690BB15069A6
:103E90009847BDE80840FEF743BD00BF3C43002003
:103EA0004FF0B04208B5D2F8883003F00803C2F8EA
:103EB000883023B1044A93690BB1D0699847BDE8B3
:103EC0000840FEF72DBD00BF3C4300204FF0B0423C
:103ED00008B5D2F8883003F01003C2F8883023B157
:103EE000044A136A0BB1506A9847BDE80840FEF7D0
:103EF00017BD00BF3C4300204FF0B04310B5D3F8CE
:103F0000884004F47872C3F88820A30604D5124AC6
:103F1000936A0BB1D06A9847600604D50E4A136BBA
:103F20000BB1506B9847210604D50B4A936B0BB12C
:103F3000D06B9847E20504D5074A136C0BB1506C5F
:103F40009847A30504D5044A936C0BB1D06C9847ED
:103F5000BDE81040FEF7E4BC3C4300204FF0B04306
:103F600010B5D3F8884004F47C42C3F88820620579
:103F700004D5164A136D0BB1506D9847230504D52F
:103F8000124A936D0BB1D06D9847E00404D50F4AE7
:103F9000136E0BB1506E9847A10404D50B4A936E73
:103FA0000BB1D06E9847620404D5084A136F0BB169
:103FB000506F9847230404D5044A936F0BB1D06F18
:103FC0009847BDE81040FEF7ABBC00BF3C43002063
:103FD00008B5FFF7B7FDBDE80840FEF7A1BC00003B
:103FE000062108B50846FDF79DFA06210720FDF7D2
:103FF00099FA06210820FDF795FA06210920FDF718
:1040000091FA06210A20FDF78DFA06211720FDF707
:1040100089FA06212820FDF785FA09217A20FDF783
:1040200081FA07213220BDE80840FDF77BBA000085
:1040300008B5FFF7ADFD00F00BF8FDF745FCFDF707
:1040400017FBFFF753FDBDE80840FFF72BBC00004E
:104050000023054A19460133102BC2E9001102F171
:104060000802F8D1704700BF3C43002010B5013969
:104070000244904201D1002005E0037811F8014F7D
:10408000A34201D0181B10BD0130F2E7034611F81E
:10409000012B03F8012B002AF9D1704753544D33FB
:1040A0003248373F3F3F0053544D3332483733781F
:1040B0002F3732780053544D3332483734332F374B
:1040C00035332F373530000001105A0003105900E6
:1040D0000120580003205600100002400800024052
:1040E0000008024000000B002800024008000240C7
:1040F0000408024006010C00400002400800024093
:104100000808024010020D0058000240080002405A
:104110000C08024016030E00700002400C00024022
:104120001008024000040F00880002400C0002400A
:104130001408024006051000A00002400C000240D6
:104140001808024010061100B80002400C0002409E
:104150001C08024016072F00100402400804024009
:1041600020080240000838002804024008040240E9
:1041700024080240060939004004024008040240B5
:1041800028080240100A3A0058040240080402407D
:104190002C080240160B3B00700402400C04024045
:1041A00030080240000C3C00880402400C0402402D
:1041B00034080240060D4400A00402400C040240F2
:1041C00038080240100E4500B80402400C040240BA
:1041D0003C080240160F460000000000ED150008E4
:1041E000D915000815160008011600080D1600085C
:1041F000F9150008E5150008D1150008211600087A
:10420000000000000100000000000000633000001A
:104210000C42000898240020A826002041726475F2
:1042200050696C6F740025424F415244252D424C19
:10423000002553455249414C250000000200000072
:10424000000000000D1800087D1800084000400024
:10425000583F0020683F00200200000000000000DE
:104260000300000000000000C51800080000000066
:1042700010000000783F0020000000000100000056
:1042800000000000EC410020010102009123000821
:10429000A12200083D23000821230008430000005C
:1042A000A442000809024300020100C032090400D0
:1042B0000001020201000524001001052401000193
:1042C000042402020524060001070582030800FFFA
:1042D00009040100020A0000000705010240000075
:1042E000070581024000000012000000F0420008B3
:1042F00012011001020000400912415700020102A0
:10430000030100000403090425424F4152442500E3
:104310004E7874505834763200303132333435367A
:104320003738394142434445460000000000000050
:10433000211A0008D91C0008851D00084000400013
:1043400024430020244300200100000034430020C7
:104350008000000040010000080000000001000093
:1043600000100000080000006D61696E0069646C57
:10437000650000005000802A00000000AAAAAAAA36
:1043800050000024FFFF00000000000000A00A0011
:104390000000004000000000AAAAAAAA0000000035
:1043A000FFFF0000000000000000000010000004FB
:1043B00000000000AAAAAAAA10000004FFFF000043
:1043C00000000000000000000000400000000000AD
:1043D000AAAAAAAA00000000FFFF00000000000037
:1043E000000000000000000000000000AAAAAAAA25
:1043F00000000000FFFF00000000000000000000BF
:104400000000000000000000AAAAAAAA0000000004
:10441000FFFF00000000000000000000000000009E
:1044200000000000AAAAAAAA00000000FFFF0000E6
:10443000000000000000000000000000000000007C
:10444000AAAAAAAA00000000FFFF000000000000C6
:10445000000000000000000000000000AAAAAAAAB4
:1044600000000000FFFF000000000000000000004E
:104470000000000000000000AAAAAAAA0000000094
:10448000FFFF00000000000000000000000000002E
:1044900000000000AAAAAAAA00000000FFFF000076
:1044A0000000000000000000870400000000000081
:1044B00000001A0000000000FF00000000000000E3
:1044C0009C40000883040000A7400008500400003E
:1044D000B5400008009600000000080096000000AB
:1044E0000008000004000000044300080000000071
:1044F00000000000000000000000000000000000BC
:0445000000000000B7
:00000001FF
